:03000000020020DB
:100020007530AC75310DE590F4F8600FC3E5302400
:1000300004F530E5313400F531D8F11200AD74C467
:1000400012006874F8120068741312006874A41225
:100050000068E531120068E53012006812009C75F6
:10006000A8817587010080B87F08334005C2B102BE
:100070000074D2B1000000D2B00000000000C2B095
:10008000DFE8D2B10000000000D2B000000030B1C3
:1000900005D201C2B02200C201C2B022C2B100002A
:1000A000000000D2B00000000000D2B122D2B0D2D5
:1000B000B10000000000C2B10000000000C2B02288
:1000C00074007F08D2B0000000A2B100C2B03300BB
:1000D000000000DFEF000000200210C2B1000000AD
:0C00E000D2B00000000000C2B0000022FE
:00000001FF
